:020000020000FC
:0200000006C038
:10000C00FDC02FED2DBF23E028BB2CEF27BB2CE729
:10001C0022BB21E021BB76D0B09B02C0B199FFC1BD
:10002C00AED0FFD0BED058EC52BF22E029BF22E0A8
:10003C0023BF7894B09919D0B1991AD0F0E0EBE6BF
:10004C0020906100109062007FD144E857D090D08E
:10005C00F0E0EFE7209075001090760075D144EC3D
:10006C004DD086D01FEF74D0E5CFF0E0E1E602C0B2
:10007C00F0E0E5E7002401920082089540E83ED0CC
:10008C00089540EC3BD008950000000000000000F3
:10009C000000000000000000000000000000000054
:1000AC000000000000000000000000000000000044
:1000BC0008954F9340E84A950000E9F74F91089551
:1000CC004F934DE11FEF1A95F1F74A95D9F74F91E0
:1000DC0008951F934F93407F486008F0446048BBDD
:1000EC00D3DF4F91C3984295407F486008F044603D
:1000FC0048BBCADFC398DDDF1F9108950894E9CF90
:10010C008894E7CF42E3DCDF4A95E9F748E348BB44
:10011C00BBDFC398D5DFD4DF48E348BBD1DF48E36E
:10012C0048BBB2DFCDDF48E2E9DF48E2E7DF48E079
:10013C00E5DF41E0E3DFC4DF46E0E0DF4EE0DEDF99
:10014C00BFDF089542E312E303D04A95E9F708951F
:10015C0023E32A9500000000E1F71A95C9F70895EA
:10016C00C895002021F0402DCBDF3196F9CF0895B2
:10017C004191442319F0C4DF4191FBCF08957EDFF8
:10018C00F1E0E0ECEDDF18ECE3DF7BDFF1E0E2ED3A
:10019C00E7DFD8DFD7DFD6DF41E0B0DF18ECD8DF00
:1001AC0008956CDFF1E0E4EEDBDF6BDFF1E0E6EF0E
:1001BC00D7DF08954469676974616C2020526561CA
:1001CC00646F7574000020286329204D2E20486F21
:1001DC006D707573202000005820202020202020D6
:1001EC002020202020202020000052202020202011
:1001FC0020202020202020202020000052BFEF9320
:10020C00FF93CF93DF93AF93BF930F930FB726D08A
:10021C000FBF0F91BF91AF91DF91CF91FF91EF91F4
:10022C00189528E240E0F0E0E0E641932140E8F741
:10023C0020E007D00093730021E003D000938700E7
:10024C000895E199FECF2EBBE09A0DB30895E19984
:10025C00FECF2EBB0DBBE29AE19A0895BB27829983
:10026C00B1608399B260E0E6F0E007D0BB278499D7
:10027C00B1608599B260E4E7F0E0A081C281D181E0
:10028C00BA17D9F0A03029F4B230B1F0B13099F0EE
:10029C0014C0A23029F4B33079F0B03061F00DC045
:1002AC00A33029F4B13041F0B23029F006C0B0309F
:1002BC0019F0B33011F422972196B083C283D18305
:1002CC00089508D006E0F02EFA9401910032E1F383
:1002DC003197089512D004E0F02E0081002329F408
:1002EC0000E20193FA94C9F70081F394005D019345
:1002FC000081FA94D9F735970895CF92DF9207E2EF
:10030C00E02E00E1F02E14D003E0E02E08EEF02EEB
:10031C000FD000E0E02E04E6F02E0AD000E0E02E34
:10032C000AE0F02E05D0D0823497DF90CF9008955C
:10033C000027CE1438F011F4DF1420F0DF18CE08AB
:10034C000395F7CF0193089501D00895208520FDE2
:10035C0008D00DD00AF405D0208521FD32D034D040
:10036C00089520941094139408F023940895E8941D
:10037C0022200AF46894089500E0602E00E0502ECC
:10038C0004E0402E00E0302EAA24992488247724FF
:10039C00012D022909F408952694179420F4730C66
:1003AC00841C951CA61C330C441C551C661CF0CFDD
:1003BC00A79497948794A79497948794292C182C96
:1003CC000895111C221C08950DE20EF00BE200831F
:1003DC0007E2402E00E1302E19D0018303E0402EBD
:1003EC0008EE302E13D00283442404E6302E0ED0B7
:1003FC0003830EE2048344240AE0302E07D00583E5
:10040C00442401E0302E02D00683089500E3131437
:10041C00240408F40895131824080395F8CF2EDE4D
:10042C00F5E0E4E39DDE2DDEF5E0E6E499DEB1993E
:10043C00FECFB099FCCF25DEF5E0E8E591DE40E893
:10044C005DDEF5E0EAE68CDE20E0FBDEB099FECF67
:10045C00B199FCCF35DE61E000FD06C044E84EDE0C
:10046C00F5E0EEE87DDE05C044E848DEF5E0ECE9B9
:10047C0077DEB19903C0B0990627E8CF0000B09998
:10048C00FECFB199FCCF1CDE62E001FD06C044E852
:10049C0035DEF5E0EAEA64DE05C044E82FDEF5E07F
:1004AC00E8EB5EDEB19903C0B0990627E8CF0000F7
:1004BC00CEDE40E823DEF5E0ECE752DE21E0C1DEE3
:1004CC00B099FECFB199FCCFFBDD61E000FD06C019
:1004DC0044E814DEF5E0EEE843DE05C044E80EDE49
:1004EC00F5E0ECE93DDEB19903C0B0990627E8CF01
:1004FC000000B099FECFB199FCCFE2DD62E001FDC6
:10050C0006C044E8FBDDF5E0EAEA2ADE05C044E873
:10051C00F5DDF5E0E8EB24DEB19903C0B0990627D0
:10052C00E8CF000094DE7CCD436F6E666967204D8A
:10053C00656E752C6472756B000020202065656EED
:10054C0020746F6574732020202000002020202050
:10055C00202020202020202020204F4B0000582D30
:10056C00617320202020202020202020202000002B
:10057C00592D617320202020202020202020202095
:10058C000000206E6F726D61616C2020203F0000B6
:10059C0020696E76657273202020203F0000204178
:1005AC00616E772E20783120203F00002041616E53
:0A05BC00772E20783220203F000047
:00000001FF
